:020000040000FA
:100000000C9463000C948B000C948B000C948B006C
:100010000C948B000C948B000C948B000C948B0034
:100020000C948B000C948B000C948B000C948B0024
:100030000C948B000C948B000C948B000C948B0014
:100040000C947D090C948B000C944B090C9425099D
:100050000C948B000C948B000C948B000C948B00F4
:100060000C948B000C948B000000000024002700EF
:100070002A000000000023002600290000000008DC
:10008000000201000003040700000000000000005F
:10009000010204081020408001020408102001021F
:1000A0000408102000000000250028002B00040494
:1000B0000404040404040202020202020303030310
:1000C0000303C7092C0D11241FBECFEFD8E0DEBFFC
:1000D000CDBF12E0A0E0B1E0E8ECF3E202C0059091
:1000E0000D92A634B107D9F723E0A6E4B2E001C02F
:1000F0001D92A033B207E1F710E0C2E6D0E004C0E1
:100100002197FE010E949810C136D107C9F70E94BD
:10011000A30A0C94D7110C9400000F931F93209105
:10012000F8023091F902232B09F44BC061157105D7
:1001300009F447C02091000330910103232B99F467
:100140004FB7F8940091570210915802209159022C
:1001500030915A024FBF0093FC021093FD0220938E
:10016000FE023093FF02E091FA02F091FB0220912F
:10017000F8023091F902232B89F02091000330918D
:1001800001032115310551F042815381452B31F096
:10019000215031093093010320930003009711F49B
:1001A00081E090E09183808393838283758364836D
:1001B0008091000390910103019690930103809335
:1001C00000031F910F910895E091FA02F091FB0254
:1001D00080819181009721F0648175810C948D005C
:1001E000089580E480937C0080917A0080648093FD
:1001F0007A0080917A0086FDFCCF80917800909102
:1002000079000895E0910F03F091100340910503E8
:10021000509106039A01220F331F240F351F2E0F12
:100220003F1FE217F30728F47083618382833396BC
:10023000F8CF809107038068809307030895209189
:100240000503309106038217930798F4FC01EE0F23
:10025000FF1F8E0F9F1FE0910F03F0911003E80F17
:10026000F91F5083418362838091070380688093E4
:1002700007030895AF92BF92CF92DF92EF92FF9261
:100280000F931F93CF93DF936C017B018B01040FBE
:10029000151FEB015E01AE18BF08C017D10759F05A
:1002A0006991D601ED91FC910190F081E02DC6019C
:1002B0000995892B79F7C501DF91CF911F910F9196
:1002C000FF90EF90DF90CF90BF90AF900895FC012A
:1002D000538D448D252F30E0842F90E0821B930BAB
:1002E000541710F0CF96089501970895FC01918D51
:1002F000828D981761F0A28DAE0FBF2FB11D5D9654
:100300008C91928D9F5F9F73928F90E008958FEFF5
:100310009FEF0895FC01918D828D981731F0828DA9
:10032000E80FF11D858D90E008958FEF9FEF089500
:10033000FC01918D228D892F90E0805C9F4F821B64
:1003400091098F73992708958BE592E00E94980197
:1003500021E0892B09F420E0822F089580E090E0CD
:10036000892B29F00E94A40181110C9400000895AA
:10037000FC01A48DA80FB92FB11DA35ABF4F2C911A
:10038000848D90E001968F739927848FA689B78911
:100390002C93A089B1898C91837080648C93938D08
:1003A000848D981306C00288F389E02D80818F7DAB
:1003B00080830895EF92FF920F931F93CF93DF9363
:1003C000EC0181E0888F9B8D8C8D98131AC0E88991
:1003D000F989808185FF15C09FB7F894EE89FF8960
:1003E0006083E889F98980818370806480839FBFFE
:1003F00081E090E0DF91CF911F910F91FF90EF90FE
:100400000895F62E0B8D10E00F5F1F4F0F7311270D
:10041000E02E8C8D8E110CC00FB607FCFACFE88948
:10042000F989808185FFF5CFCE010E94B801F1CF17
:10043000EB8DEC0FFD2FF11DE35AFF4FF0829FB7BC
:10044000F8940B8FEA89FB8980818062CFCFCF93AC
:10045000DF93EC01888D8823B9F0AA89BB89E889EC
:10046000F9898C9185FD03C0808186FD0DC00FB692
:1004700007FCF7CF8C9185FFF2CF808185FFEDCF10
:10048000CE010E94B801E9CFDF91CF91089583306A
:1004900081F028F4813099F08230A9F008958730F6
:1004A000A9F08830C9F08430B1F4809180008F7D4C
:1004B00003C0809180008F7780938000089584B579
:1004C0008F7784BD089584B58F7DFBCF8091B00078
:1004D0008F778093B00008958091B0008F7DF9CF21
:1004E000CF93DF9390E0FC01E057FF4F24918255BA
:1004F0009F4FFC0184918823C9F090E0880F991FD9
:10050000FC01E859FF4FA591B491FC01EC55FF4F58
:10051000C591D49161110DC09FB7F8948C9120952D
:1005200082238C938881282328839FBFDF91CF91DA
:100530000895623051F49FB7F8943C91822F8095D2
:1005400083238C93E8812E2BEFCF8FB7F894EC9117
:100550002E2B2C938FBFEACF3FB7F89480914D029A
:1005600090914E02A0914F02B091500226B5A89BE7
:1005700005C02F3F19F00196A11DB11D3FBFBA2F35
:10058000A92F982F8827BC01CD01620F711D811DF5
:10059000911D42E0660F771F881F991F4A95D1F77A
:1005A00008950F931F93CF93DF9300D000D000D016
:1005B0001F92CDB7DEB78091070387FF66C00E9408
:1005C000AC0200910B0310910C0320910D033091AC
:1005D0000E03601B710B820B930B6C327140810513
:1005E000910568F3F89480911303E0911103F09161
:1005F0001203409108035091090320910F03309199
:1006000010035A83498389010F5F1F4FD9019C91C1
:100610009F839081982B9E839081809589238D83E1
:100620008D818C8388E08B835E816D814F813B81DE
:100630002C8189819A81D801508347FD252F3A95D5
:100640002083262F39F0441F00C000006083000083
:1006500000C0F2CF38E04D9160830000019761F750
:100660004F833B832C839A83898378940E94AC02C6
:1006700060930B0370930C0380930D0390930E0310
:10068000809107038F778093070327960FB6F8941E
:10069000DEBF0FBECDBFDF91CF911F910F910895A7
:1006A0008F929F92AF92BF92CF92DF92EF92FF9282
:1006B0004B015C010E94AC026B017C010E94AC0208
:1006C0006C197D098E099F09683E7340810591056B
:1006D000A8F321E0821A9108A108B10888EEC80E9B
:1006E00083E0D81EE11CF11C81149104A104B10423
:1006F00029F7FF90EF90DF90CF90BF90AF909F9041
:100700008F9008952F923F924F925F926F927F92B7
:100710008F929F92AF92BF92CF92DF92EF92FF9211
:100720000F931F93CF93DF933B014C015901D42FBB
:10073000C52F6701780120E030E0A901C801B601AA
:100740000E94B30E87FF0AC020E030E040E85FE37C
:10075000C801B6010E94470E6B017C0120E030E029
:1007600040E85FE3C701B6010E941210181654F466
:1007700020E030E040E85FE3C701B6010E94460E8A
:100780006B017C012BEA3AEA4AE25EE3C701B6015B
:100790000E94B30E87FF2EC09301A401B5018D2FD7
:1007A0009C2F0E94460E20E030E040EC50E40E9476
:1007B0001710A70196010E9417109301A4010E942F
:1007C000470E5B01D82FC92FB5018D2F9C2FDF91CC
:1007D000CF911F910F91FF90EF90DF90CF90BF903E
:1007E000AF909F908F907F906F905F904F903F90D1
:1007F0002F90089520E030E040E05FE3C701B601AC
:100800000E94B30E87FDE0CF2BEA3AEA4AE25FE3AB
:10081000C701B6010E94B30E87FF1CC09301A4015B
:10082000B5018D2F9C2F0E94460E1B012C01A701A4
:1008300096016BEA7AEA8AE29FE30E94460E9B01E8
:10084000AC01C201B1010E94171020E030E040EC81
:1008500050E4B1CF5301D82DC92DB6CF2F923F927E
:100860004F925F926F927F928F929F92AF92BF92C0
:10087000CF92DF92EF92FF920F931F93CF93DF936C
:10088000CDB7DEB72A970FB6F894DEBF0FBECDBF47
:100890001C01FB0180819181A281B38189839A83AC
:1008A000AB83BC8384809580A680B78090859A872F
:1008B000A185A987D284C38420E030E0A901C501C5
:1008C000B4010E94B30E882309F4C9C020E030E0CF
:1008D000A9016A8579858D2D9C2D0E94B30E8823F0
:1008E00009F4BDC020E030E040E05FE36A8579852F
:1008F0008D2D9C2D0E94B30E87FF98C020E030E024
:1009000040E85FE3C501B4010E94470E2A8539859E
:100910004D2D5C2D0E9417104B015C012A853985F5
:100920004D2D5C2D6A8579858D2D9C2D0E94470E5D
:10093000A50194010E94460E2B013C012BEA3AEAE4
:100940004AEA5EE369817A818B819C810E94470E2D
:100950007B018C01A5019401C301B2010E948203B5
:100960006A877987D82EC92EE980FA800B811C818D
:10097000A5019401C301B2010E9482036D837E83AD
:100980008F8398872BEA3AEA4AEA5EE3C801B70107
:100990000E94460E7B018C01A5019401C301B201A6
:1009A0000E9482034B015C0120E030E04FE753E4FA
:1009B0006A8579858D2D9C2D0E9417100E94310F1C
:1009C000F101608320E030E04FE753E46D817E81E8
:1009D0008F8198850E9417100E94310FD1011196C6
:1009E0006C9320E030E04FE753E4B401C5010E946E
:1009F00017100E94310FF10162832A960FB6F89406
:100A0000DEBF0FBECDBFDF91CF911F910F91FF9041
:100A1000EF90DF90CF90BF90AF909F908F907F909E
:100A20006F905F904F903F902F9008952A85398561
:100A30004D2D5C2DC501B4010E94470E2B013C01D8
:100A40002A8539854D2D5C2DC501B4010E941710F2
:100A50009B01AC01C301B2010E94460E5DCF8A84A6
:100A60009984AD2CBC2C8D829E82DF82C8869CCF5F
:100A70002F923F924F925F926F927F928F92AF929E
:100A8000BF92CF92DF92EF92FF920F931F93CF937B
:100A9000DF937C0120E030E048EC52E4FC0160810F
:100AA0007181828193810E9417100E942A0F5B013D
:100AB0006091290370912A0380912B030E94020107
:100AC0008091480290914902833C910584F0809185
:100AD00046029091470210924902109248020196F4
:100AE0008730910554F59093470280934602809198
:100AF00046029091470260902003709021038090FD
:100B0000220383309105C1F1ECF4609017037090DB
:100B10001803809019038130910571F160901D03D5
:100B200070901E0380901F03029731F1609026039E
:100B300070902703809028031FC0109247021092E4
:100B40004602D5CF60902303709024038090250344
:100B50008530910589F060901A0370901B03809096
:100B60001C038530910544F06090140370901503C8
:100B7000809016030697D1F6D0E0C0E08CE7482EAF
:100B80005524539496E6292E3324339406E411E039
:100B9000C0904802D0904902C6018C0F9D1F833C33
:100BA00091055CF4682DA301853591058CF50E94B3
:100BB0001F012196C630D10559F7C50163E070E0E9
:100BC0000E948410892B31F4C6010196909349024A
:100BD00080934802F701868197810297C9F5809139
:100BE000F8029091F902892B99F1DF91CF911F9131
:100BF0000F91FF90EF90DF90CF90BF90AF908F90CC
:100C00007F906F905F904F903F902F900C94E400F6
:100C100022EC30E08F36910594F0E4EFF0E0873875
:100C2000910594F020E231E08B39910544F0F80110
:100C30008D3A91054CF08B3B91052CF49101281BCA
:100C4000390BC901B4CFF201E81BF90BCF01AFCFCB
:100C5000DF91CF911F910F91FF90EF90DF90CF9098
:100C6000BF90AF908F907F906F905F904F903F902C
:100C70002F9008958091F8029091F902892B11F03C
:100C80000C94E40008950F931F93CF93DF93CDB797
:100C9000DEB72F970FB6F894DEBF0FBECDBF8C0125
:100CA000FC0180819181A281B38189839A83AB8386
:100CB000BC8380E090E0A0E8BFE38D839E83AF8398
:100CC000B8878DEC9CECACE4BDE389879A87AB8751
:100CD000BC87BE016F5F7F4FCE010D960E942E0430
:100CE0006D857E858F850E940201F801868197813E
:100CF000029711F40E943A062F960FB6F894DEBFC1
:100D00000FBECDBFDF91CF911F910F9108952F920C
:100D10003F924F925F926F927F928F92BF92CF924B
:100D2000DF92EF92FF920F931F93CF93DF938A315D
:100D300008F051C03A01862E08E212E0D0E0C0E08F
:100D4000C82ED12CF12CE12C8AE1B82EF80161914A
:100D50008F0170E090E080E00E94600F20E030E0C2
:100D600040ED51E40E94B80E1B012C01C701B601F1
:100D70000E94620F9B01AC01C201B1010E941710D9
:100D80001B012C0120E030E0A9010E94121020E09C
:100D900030E040E05FE387FD2FC0C201B1010E9457
:100DA000470E0E942A0FBC9EC001BD9E900D1124CB
:100DB000865F9E4F680F791FFB018081882331F089
:100DC000682DA3018150990B0E941F012196CB3001
:100DD000D10509F0BBCFDF91CF911F910F91FF900B
:100DE000EF90DF90CF90BF908F907F906F905F904B
:100DF0004F903F902F900895C201B1010E94460E7E
:100E0000D0CF4F925F926F927F92AF92BF92CF926C
:100E1000DF92EF92FF920F931F93CF93DF93CDB7A3
:100E2000DEB72F970FB6F894DEBF0FBECDBF5C01C3
:100E300010E000E08DEC482E8CEC582E8CE4682EEF
:100E40008DE3782EB801012E000C880B990B0E94BF
:100E5000620F20E030E040ED51E40E94B80EF50151
:100E600020813181428153810E94470E6B017C01B8
:100E700020E030E040E85FE30E941210181654F4BE
:100E800020E030E040E85FE3C701B6010E94460E73
:100E90006B017C01C982DA82EB82FC8280E090E007
:100EA000A0E8BFE38D839E83AF83B88749865A86C7
:100EB0006B867C86BE016F5F7F4FCE010D960E94D0
:100EC0002E044D855E856F85802F0E9487060F5FFB
:100ED0001F4F0A31110509F0B5CFF50186819781C1
:100EE000029711F40E943A062F960FB6F894DEBFCF
:100EF0000FBECDBFDF91CF911F910F91FF90EF906B
:100F0000DF90CF90BF90AF907F906F905F904F90A9
:100F10000895CF93DF93EC0120E030E048ED51E4F9
:100F2000688179818A819B810E9417100E942A0F13
:100F3000CB016A3171056CF020914A0230914B026D
:100F40002F5F3F4F27303105B4F430934B0220938D
:100F50004A02E0914A02F0914B02E730F105C0F4F9
:100F6000EC54F84F0C949810C007D607DD07E4073F
:100F7000EB07F207F90710924B0210924A02E9CFF1
:100F80004091260350912703609128030E94870611
:100F90008E819F810297A1F58091F8029091F902CC
:100FA000892B71F1DF91CF910C94E40040912303E0
:100FB0005091240360912503E9CF40912003509183
:100FC000210360912203E2CF40911D0350911E0343
:100FD00060911F03DBCF40911A0350911B03609176
:100FE0001C03D4CF4091170350911803609119034B
:100FF000CDCF409114035091150360911603C6CFD5
:10100000DF91CF9108952F923F924F925F926F920E
:101010007F928F929F92AF92BF92CF92DF92EF9288
:10102000FF920F931F93CF93DF93CDB7DEB72F9728
:101030000FB6F894DEBF0FBECDBF5C018AE0C82EAC
:1010400081E0D82E10E000E09DEC292E9CEC392E9A
:101050009CE4492E9DE3592EB801012E000C880B0B
:10106000990B0E94620F20E030E040E351E40E94BF
:10107000B80EF50120813181428153810E94470ED3
:101080003B014C0120E030E040E85FE30E94121099
:10109000181654F420E030E040E85FE3C401B301E7
:1010A0000E94460E3B014C0169827A828B829C82AF
:1010B00080E090E0A0E8BFE38D839E83AF83B88794
:1010C00029863A864B865C86BE016F5F7F4FCE01D4
:1010D0000D960E942E046D847E848F84F12CE12C69
:1010E000F601EE0DFF1D8081882369F0682DA301B4
:1010F0008150990B0E941F01FFEFEF1AFF0A8AE14E
:10110000E816F10469F70F5F1F4FEAE1CE0ED11C1C
:101110000B30110509F0A0CFF50186819781029768
:1011200011F40E943A062F960FB6F894DEBF0FBE58
:10113000CDBFDF91CF911F910F91FF90EF90DF9086
:10114000CF90BF90AF909F908F907F906F905F9067
:101150004F903F902F9008954F925F926F927F92A1
:101160008F929F92AF92BF92CF92DF92EF92FF92B7
:101170000F931F93CF93DF93CDB7DEB72F970FB6A3
:10118000F894DEBF0FBECDBFFC0186819781029728
:1011900009F044C010E000E088EE482E83E0582EAD
:1011A000612C712C812C912C90E8A92E9FE3B92EF3
:1011B0002DECC22E2CECD22E2CE4E22E2DE3F22EBE
:1011C0000E948B0DA30192010E94E30D0E94620F09
:1011D00020E030E04AE754E40E94B80E69837A8345
:1011E0008B839C838D829E82AF82B886C986DA8685
:1011F000EB86FC86BE016F5F7F4FCE010D960E948D
:101200002E044D855E856F85C8010E941F010F5F0A
:101210001F4F023C1105A1F60E943A062F960FB609
:10122000F894DEBF0FBECDBFDF91CF911F910F911C
:10123000FF90EF90DF90CF90BF90AF909F908F90F6
:101240007F906F905F904F9008951F920F920FB60E
:101250000F9211242F933F934F935F936F937F933C
:101260008F939F93AF93BF93EF93FF938BE592E0A0
:101270000E94B801FF91EF91BF91AF919F918F9123
:101280007F916F915F914F913F912F910F900FBE82
:101290000F901F9018951F920F920FB60F92112466
:1012A0002F938F939F93EF93FF93E0916B02F091B5
:1012B0006C028081E0917102F091720282FD1BC08C
:1012C0009081809174028F5F8F73209175028217D5
:1012D00041F0E0917402F0E0E55AFD4F958F809364
:1012E0007402FF91EF919F918F912F910F900FBEFC
:1012F0000F901F9018958081F4CF1F920F920FB618
:101300000F9211242F933F938F939F93AF93BF938B
:101310008091570290915802A0915902B0915A02BF
:1013200030914C0223E0230F2D3758F50196A11D73
:10133000B11D20934C028093570290935802A093C2
:101340005902B0935A0280914D0290914E02A091A1
:101350004F02B09150020196A11DB11D80934D0224
:1013600090934E02A0934F02B0935002BF91AF9161
:101370009F918F913F912F910F900FBE0F901F90D3
:10138000189526E8230F0296A11DB11DD2CF109209
:101390005E0210925D0288EE93E0A0E0B0E08093E0
:1013A0005F0290936002A0936102B093620287E3B0
:1013B00092E090935C0280935B0285EC90E09093C6
:1013C00068028093670284EC90E090936A028093B5
:1013D000690280EC90E090936C0280936B0281EC48
:1013E00090E090936E0280936D0222EC30E0309397
:1013F000700220936F0286EC90E0909372028093CB
:10140000710210927402109275021092760210927C
:1014100077021092290310922A0310922B03109244
:1014200026038CE380932703109228039CE090937B
:10143000230380932403109225039EE190932003BD
:10144000909321031092220380931D0310921E0398
:1014500010921F0390931A0310921B0380931C0396
:10146000109217031092180380931903109214031B
:10147000909315038093160330930603209305037E
:101480001092070386E492E0909309038093080387
:1014900083E180930A0310921203109211031092B9
:1014A000130361E00E947002809108039091090388
:1014B0000E94B2109093100380930F03E1ECF0E0D0
:1014C000E491F0E0EE0FFF1FEC55FF4F85919491F2
:1014D0009093120380931103E3EAF0E0E491E09328
:1014E00013038AE090E09093F9028093F80210923F
:1014F000FC021092FD021092FE021092FF02109266
:1015000001031092000381E08093040381E090E0E6
:1015100090930303809302038CE390E00E94B21047
:10152000FC019C01245C3F4F1182108213821282C5
:10153000158214823696E217F307B1F79093FB02F7
:101540008093FA020895CF93DF93CDB7DEB72E973D
:101550000FB6F894DEBF0FBECDBF789484B582601D
:1015600084BD84B5816084BD85B5826085BD85B547
:10157000816085BD80916E00816080936E001092C5
:101580008100809181008260809381008091810040
:1015900081608093810080918000816080938000D1
:1015A0008091B10084608093B1008091B00081602F
:1015B0008093B00080917A00846080937A0080915B
:1015C0007A00826080937A0080917A0081608093B3
:1015D0007A0080917A00806880937A001092C1002E
:1015E00062E08EE00E947002E0916B02F0916C026A
:1015F00082E08083E0916702F09168021082E091BE
:101600006902F0916A0280E1808310927302E09196
:101610006F02F091700286E08083E0916D02F0919C
:101620006E02808180618083E0916D02F0916E0294
:10163000808188608083E0916D02F0916E028081EC
:1016400080688083E0916D02F0916E0280818F7DD1
:1016500080830E94F1006C01990FEE08FF0861E0A1
:1016600070E080E090E00E94500303E010E00E94F0
:10167000F100002E02C0880F991F0A94E2F74C0176
:10168000990FAA08BB08240135014C245D246E245F
:101690007F2461E070E080E090E00E9450030D5FE5
:1016A0001F4F0132110509F0E1C08C149D04AE04F6
:1016B000BF0421F0C301B2010E94DA0D20910A0398
:1016C00030E0F901E458FF4F8491F901E057FF4FF2
:1016D0000491F901E255FF4F1491112391F081110A
:1016E0000E944702E12FF0E0EE0FFF1FEC55FF4F85
:1016F000A591B4918FB7F894EC9100950E230C93BB
:101700008FBF0E94AC0260930B0370930C03809315
:101710000D0390930E0360E070E080E00E940201F0
:101720006091290370912A0380912B030E9402018A
:101730000E94D10280910403882309F4C4C08FB7AA
:10174000F894C0905702D0905802E0905902F0905F
:101750005A028FBF8091FC029091FD02A091FE027F
:10176000B091FF02A7019601281B390B4A0B5B0BB6
:10177000CA01B901209102033091030350E040E017
:10178000621773078407950708F49DC00E94150E21
:1017900049015A011C861B8610E000E08091F80286
:1017A0009091F9020817190708F085C02090FA02F5
:1017B0003090FB024B855C85240E351ED1011496BA
:1017C0000D90BC91A02DBE87AD871E830D83F101C6
:1017D00082819381AC0170E060E084169506A606D4
:1017E000B70608F046C0208131813A87298721E079
:1017F00030E049855A858417950711F430E020E0E0
:1018000038872F8369857A85681B790B90E080E0A3
:101810000E94600F2B013C01A985BA85BD0190E0B3
:1018200080E00E94600F9B01AC01C301B2010E94E5
:10183000B80E69837A838B839C83CE010196ED85F4
:10184000FE850995D10112968D919C911397881967
:10185000990913969C938E9312970F5F1F4F2B85B8
:101860003C852A5F3F4F3C872B8798CF73016201ED
:10187000FECE892B91F3E2E0F0E0F887EF8320E0E1
:1018800030E040E85FE329833A834B835C838091B7
:10189000000390910103019790930103809300034B
:1018A000D10113961C921E921297CE010196ED85DE
:1018B000FE850995D2CFC092FC02D092FD02E09243
:1018C000FE02F092FF020E94D1026AE070E080E026
:1018D00090E00E945003EAE8F0E08491EEE9F0E045
:1018E0001491ECEBF0E00491002309F45DC0811148
:1018F0000E944702E02FF0E0EE0FFF1FEE58FF4F6F
:10190000A591B4918C91182309F44EC08091530293
:1019100090915402A0915502B09156020097A105F2
:10192000B10509F05CC02FB7F894809157029091EF
:101930005802A0915902B0915A022FBF80935302CE
:1019400090935402A0935502B09356028091510295
:10195000909152028230910509F46FC084F400978F
:1019600009F45FC0019709F463C08091510290911E
:1019700052020196909352028093510245C08430E6
:10198000910509F464C00CF45DC0059771F76CEA29
:1019900078E084E690E00E948D008FEF9FEF9093B7
:1019A000520280935102E1CF609126037091270388
:1019B000809128030E9402010E94D10268EE73E028
:1019C00080E090E00E9450036091290370912A0307
:1019D00080912B030E9402010E94D102FFCF2FB7FA
:1019E000F8944091570250915802609159027091B9
:1019F0005A022FBF8857934DAF4FBF4F841795079B
:101A0000A607B70708F48FCF80E090E0892B09F490
:101A100091CE0E94A401882309F48CCE0E9400007C
:101A200089CE68E375E084EF91E00E948D009DCF40
:101A300069E877E088E592E0F8CF61E077E088EB4D
:101A40009BE0F3CF63E078E080ED97E0EECF63E4D6
:101A500076E080E49FE1E9CF8091FA029091FB0269
:101A6000009711F00E944E1160E080910A030E94DD
:101A7000700280910F03909110030C944E118F927D
:101A80009F92AF92BF92CF92DF92EF92FF92CF934D
:101A9000DF93EC01688179818A819B8161157105F1
:101AA0008105910521F464E279ED8BE597E02DE164
:101AB00033EF41E050E00E94E30D49015A019B01E0
:101AC000AC01A7EAB1E40E94020E6B017C01ACEE0E
:101AD000B4EFA50194010E94100EC60ED71EE81E99
:101AE000F91EF7FE06C081E0C81AD108E10880E8B7
:101AF000F80AC882D982EA82FB82C701B6019F77C1
:101B0000DF91CF91FF90EF90DF90CF90BF90AF909B
:101B10009F908F9008958F929F92AF92BF92CF9295
:101B2000DF92EF92FF92609100017091010180912C
:101B3000020190910301611571058105910521F460
:101B400064E279ED8BE597E02DE133EF41E050E081
:101B50000E94E30D49015A019B01AC01A7EAB1E4DF
:101B60000E94020E6B017C01ACEEB4EFA501940162
:101B70000E94100EC60ED71EE81EF91EF7FE06C004
:101B800081E0C81AD108E10880E8F80AC092000193
:101B9000D0920101E0920201F0920301C701B60167
:101BA0009F77FF90EF90DF90CF90BF90AF909F9086
:101BB0008F9008956093000170930101809302015A
:101BC000909303010895052E97FB1EF400940E9444
:101BD000FA0D57FD07D00E94150E07FC03D04EF4F6
:101BE0000C94FA0D50954095309521953F4F4F4FED
:101BF0005F4F089590958095709561957F4F8F4FB9
:101C00009F4F08950E94370EA59F900DB49F900D91
:101C1000A49F800D911D11240895B7FF0C94020E0E
:101C20000E94020E821B930B0895A1E21A2EAA1B9A
:101C3000BB1BFD010DC0AA1FBB1FEE1FFF1FA2177C
:101C4000B307E407F50720F0A21BB30BE40BF50B79
:101C5000661F771F881F991F1A9469F76095709502
:101C6000809590959B01AC01BD01CF010895A29F85
:101C7000B001B39FC001A39F700D811D1124911D60
:101C8000B29F700D811D1124911D08955058BB27DE
:101C9000AA270E945E0E0C94D80F0E94CA0F38F03B
:101CA0000E94D10F20F039F49F3F19F426F40C94D0
:101CB000C70F0EF4E095E7FB0C94C10FE92F0E94CB
:101CC000E90F58F3BA17620773078407950720F0E6
:101CD00079F4A6F50C940B100EF4E0950B2EBA2FA8
:101CE000A02D0B01B90190010C01CA01A001112422
:101CF000FF27591B99F0593F50F4503E68F11A16CE
:101D0000F040A22F232F342F4427585FF3CF46955E
:101D100037952795A795F0405395C9F77EF41F1680
:101D2000BA0B620B730B840BBAF09150A1F0FF0F4A
:101D3000BB1F661F771F881FC2F70EC0BA0F621F36
:101D4000731F841F48F4879577956795B795F79526
:101D50009E3F08F0B0CF9395880F08F09927EE0FBB
:101D60009795879508950E949D0F08F481E0089546
:101D70000E94CC0E0C94D80F0E94D10F58F00E94F4
:101D8000CA0F40F029F45F3F29F00C94C10F5111A4
:101D90000C940C100C94C70F0E94E90F68F3992360
:101DA000B1F3552391F3951B550BBB27AA27621757
:101DB0007307840738F09F5F5F4F220F331F441F64
:101DC000AA1FA9F335D00E2E3AF0E0E832D0915098
:101DD0005040E695001CCAF72BD0FE2F29D0660F85
:101DE000771F881FBB1F261737074807AB07B0E8C8
:101DF00009F0BB0B802DBF01FF2793585F4F3AF0CE
:101E00009E3F510578F00C94C10F0C940C105F3F6D
:101E1000E4F3983ED4F3869577956795B795F79553
:101E20009F5FC9F7880F911D9695879597F908953B
:101E3000E1E0660F771F881FBB1F621773078407D7
:101E4000BA0720F0621B730B840BBA0BEE1F88F7E6
:101E5000E09508950E94310F6894B1110C940C1014
:101E600008950E94F10F88F09F5798F0B92F992795
:101E7000B751B0F0E1F0660F771F881F991F1AF075
:101E8000BA95C9F714C0B13091F00E940B10B1E0BF
:101E900008950C940B10672F782F8827B85F39F0BE
:101EA000B93FCCF3869577956795B395D9F73EF40E
:101EB00090958095709561957F4F8F4F9F4F0895B6
:101EC000E89409C097FB3EF49095809570956195D4
:101ED0007F4F8F4F9F4F9923A9F0F92F96E9BB278A
:101EE0009395F695879577956795B795F111F8CF06
:101EF000FAF4BB0F11F460FF1BC06F5F7F4F8F4F71
:101F00009F4F16C0882311F096E911C0772321F066
:101F10009EE8872F762F05C0662371F096E8862FFE
:101F200070E060E02AF09A95660F771F881FDAF755
:101F3000880F9695879597F90895990F0008550F82
:101F4000AA0BE0E8FEEF16161706E807F907C0F03F
:101F500012161306E407F50798F0621B730B840B47
:101F6000950B39F40A2661F0232B242B252B21F421
:101F700008950A2609F4A140A6958FEF811D811DC1
:101F8000089597F99F6780E870E060E008959FEFFB
:101F900080EC089500240A94161617061806090600
:101FA000089500240A9412161306140605060895CF
:101FB000092E0394000C11F4882352F0BB0F40F457
:101FC000BF2B11F460FF04C06F5F7F4F8F4F9F4F97
:101FD000089557FD9058440F551F59F05F3F71F019
:101FE0004795880F97FB991F61F09F3F79F0879580
:101FF0000895121613061406551FF2CF4695F1DF09
:1020000008C0161617061806991FF1CF8695710598
:10201000610508940895E894BB2766277727CB01CC
:1020200097F908950E949D0F08F48FEF08950E947C
:102030002A100C94D80F0E94CA0F38F00E94D10FBA
:1020400020F0952311F00C94C10F0C94C70F1124AC
:102050000C940C100E94E90F70F3959FC1F3950F3B
:1020600050E0551F629FF001729FBB27F00DB11D1C
:10207000639FAA27F00DB11DAA1F649F6627B00DAC
:10208000A11D661F829F2227B00DA11D621F739F95
:10209000B00DA11D621F839FA00D611D221F749FA3
:1020A0003327A00D611D231F849F600D211D822FEA
:1020B000762F6A2F11249F5750409AF0F1F0882311
:1020C0004AF0EE0FFF1FBB1F661F771F881F91503E
:1020D0005040A9F79E3F510580F00C94C10F0C941D
:1020E0000C105F3FE4F3983ED4F38695779567959F
:1020F000B795F795E7959F5FC1F7FE2B880F911D68
:102100009695879597F9089597FB072E16F40094F6
:1021100007D077FD09D00E949E1007FC05D03EF441
:10212000909581959F4F0895709561957F4F089583
:10213000EE0FFF1F0590F491E02D0994AA1BBB1B25
:1021400051E107C0AA1FBB1FA617B70710F0A61BB7
:10215000B70B881F991F5A95A9F780959095BC01D8
:10216000CD0108950F931F93CF93DF938230910594
:1021700010F482E090E0E0912E03F0912F0330E024
:1021800020E0B0E0A0E0309799F42115310509F482
:102190004AC0281B390B24303105D8F58A819B8130
:1021A0006115710589F1FB0193838283FE0111C0E2
:1021B000408151810281138148175907E0F0481787
:1021C000590799F4109761F012960C931297139691
:1021D0001C933296CF01DF91CF911F910F910895FB
:1021E00000932E0310932F03F4CF2115310551F0E6
:1021F0004217530738F0A901DB019A01BD01DF0145
:10220000F801C1CFEF01F9CF90932F0380932E03F4
:10221000CDCFFE01E20FF31F81939193225031093C
:1022200039832883D7CF20912C0330912D03232B82
:1022300041F4209106013091070130932D03209342
:102240002C0320910401309105012115310541F441
:102250002DB73EB74091080150910901241B350B61
:10226000E0912C03F0912D03E217F307A0F42E1B4D
:102270003F0B2817390778F0AC014E5F5F4F2417EA
:10228000350748F04E0F5F1F50932D0340932C03EA
:10229000819391939FCFF0E0E0E09CCFCF93DF93C9
:1022A0000097E9F0FC01329713821282A0912E036D
:1022B000B0912F03ED0130E020E01097A1F42081D0
:1022C0003181820F931F20912C0330912D03281709
:1022D000390709F061C0F0932D03E0932C03DF91DF
:1022E000CF910895EA01CE17DF07E8F54A815B81B7
:1022F0009E0141155105B1F7E901FB83EA8349913C
:102300005991C40FD51FEC17FD0761F480819181AD
:102310000296840F951FE9019983888382819381B6
:102320009B838A83F0E0E0E012968D919C91139755
:102330000097B9F52D913C911197CD010296820F2E
:10234000931F20912C0330912D032817390739F65C
:10235000309751F510922F0310922E03B0932D0356
:10236000A0932C03BCCFD383C28340815181840FBF
:10237000951FC817D90761F44E5F5F4F8881998117
:10238000480F591F518340838A819B8193838283A5
:102390002115310509F0B0CFF0932F03E0932E0300
:1023A0009ECFFD01DC01C0CF13821282D7CF10E097
:1023B000C2E6D0E004C0FE010E9498102196C33608
:1023C000D107C9F7F894FFCF0100000000003003E7
:1023D0008000C2C1C0BFBEBDBCBB00000000000089
:1023E000000000000000000000000000BAB9B8B70B
:1023F000B6B5B4B3B2B1B0AFAEAD000000000000EE
:10240000000000000000ACABAAA9A8A7A6A5A4A341
:10241000A2A1A09F9E9D9C9B0000000000000000C8
:102420009A999897969594939291908F8E8D8C8B84
:102430008A89888700000000000086858483828165
:10244000807F7E7D7C7B7A79787776757473727104
:10245000706F00006E6D6C6B6A69686766656463B7
:102460006261605F5E5D5C5B5A59585756553D3EF0
:102470003F404142434445464748494A4B4C4D4EF4
:102480004F50515253540000292A2B2C2D2E2F30FF
:102490003132333435363738393A3B3C00000000AE
:1024A00000001718191A1B1C1D1E1F20212223248F
:1024B000252627280000000000000000090A0B0C58
:1024C0000D0E0F101112131415160000000000005D
:1024D00000000000000001020304050607080000D8
:1024E00000000000000000000000000000000000EC
:1024F000080E1214181A1814120E0800000000DA40
:0E250000013A0167012702980176018A010065
:107E0000112484B714BE81FFF0D085E080938100F7
:107E100082E08093C00088E18093C10086E0809377
:107E2000C20080E18093C4008EE0C9D0259A86E02C
:107E300020E33CEF91E0309385002093840096BBD3
:107E4000B09BFECF1D9AA8958150A9F7CC24DD24C4
:107E500088248394B5E0AB2EA1E19A2EF3E0BF2EE7
:107E6000A2D0813461F49FD0082FAFD0023811F036
:107E7000013811F484E001C083E08DD089C08234E0
:107E800011F484E103C0853419F485E0A6D080C0E4
:107E9000853579F488D0E82EFF2485D0082F10E0AE
:107EA000102F00270E291F29000F111F8ED06801E7
:107EB0006FC0863521F484E090D080E0DECF843638
:107EC00009F040C070D06FD0082F6DD080E0C81688
:107ED00080E7D80618F4F601B7BEE895C0E0D1E017
:107EE00062D089930C17E1F7F0E0CF16F0E7DF06D8
:107EF00018F0F601B7BEE89568D007B600FCFDCFD4
:107F0000A601A0E0B1E02C9130E011968C91119780
:107F100090E0982F8827822B932B1296FA010C0160
:107F200087BEE89511244E5F5F4FF1E0A038BF0790
:107F300051F7F601A7BEE89507B600FCFDCF97BE46
:107F4000E89526C08437B1F42ED02DD0F82E2BD052
:107F50003CD0F601EF2C8F010F5F1F4F84911BD097
:107F6000EA94F801C1F70894C11CD11CFA94CF0C13
:107F7000D11C0EC0853739F428D08EE10CD085E9AC
:107F80000AD08FE07ACF813511F488E018D01DD067
:107F900080E101D065CF982F8091C00085FFFCCF94
:107FA0009093C60008958091C00087FFFCCF809118
:107FB000C00084FD01C0A8958091C6000895E0E648
:107FC000F0E098E1908380830895EDDF803219F02E
:107FD00088E0F5DFFFCF84E1DECF1F93182FE3DFCA
:107FE0001150E9F7F2DF1F91089580E0E8DFEE27F6
:047FF000FF270994CA
:027FFE00040479
:00000001FF
